:100000000C94A3000C94CB000C94CB000C94CB006C
:100010000C94CB000C94CB000C94CB000C94CB0034
:100020000C94CB000C94CB000C94CB000C94CB0024
:100030000C94CB000C94CB000C94CB000C94CB0014
:100040000C94C7010C94CB000C94CB000C94CB0007
:100050000C94CB000C94CB000C94CB000C94CB00F4
:100060000C94CB000C94CB0007634236B79BD8A707
:100070001A39685618AEBAAB558C1D3CB7CC5763CD
:10008000BD6DEDFD753EF6177231BF000000803F7B
:1000900008000000BE922449123EABAAAA2ABECD97
:1000A000CCCC4C3E00000080BEABAAAAAA3E000009
:1000B0000000BF000000803F000000000008417801
:1000C000D3BB4387D1133D190E3CC3BD4282AD2B38
:1000D0003E68EC8276BED98FE1A93E4C80EFFFBE30
:1000E00001C4FF7F3F00000000000000000023006B
:1000F0002600290000000000240027002A0000003C
:100100000000250028002B00040404040404040457
:1001100002020202020203030303030301020408B2
:100120001020408001020408102001020408102061
:1001300000000008000201000003040700000000A6
:10014000000000000E0511241FBECFEFD8E0DEBF77
:10015000CDBF11E0A0E0B1E0E8EEF3E102C0059010
:100160000D92AC30B107D9F721E0ACE0B1E001C0AD
:100170001D92A233B207E1F710E0C3EAD0E004C059
:100180002197FE010E94EC09C23AD107C9F70E94EB
:1001900011020C94F2090C940000833081F028F4D1
:1001A000813099F08230A9F008958730A9F0883025
:1001B000C9F08430B1F4809180008F7D03C08091BC
:1001C00080008F7780938000089584B58F7784BDF9
:1001D000089584B58F7DFBCF8091B0008F77809399
:1001E000B00008958091B0008F7DF9CF1F93CF9319
:1001F000DF93282F30E0F901E05DFE4F8491F90193
:10020000E45EFE4FD491F901E85FFE4FC491CC2328
:10021000A9F0162F81110E94CD00EC2FF0E0EE0F17
:10022000FF1FE250FF4FA591B4918FB7F894EC9166
:10023000111108C0D095DE23DC938FBFDF91CF91E1
:100240001F910895DE2BF8CFCF93DF9390E0FC0150
:10025000E45EFE4F2491885F9E4FFC0184918823C9
:10026000D1F090E0880F991FFC01EC50FF4FA59151
:10027000B491FC01E250FF4FC591D491623071F40A
:100280009FB7F8943C91822F809583238C93E881CB
:100290002E2B28839FBFDF91CF9108958FB7F894BD
:1002A000EC912E2B2C938FBFF6CF1F93CF93DF9320
:1002B000182FEB0161E00E942401209739F460E0DF
:1002C000812FDF91CF911F910C94F600CF3FD10584
:1002D00011F461E0F5CFE12FF0E0E05DFE4FE49135
:1002E000E33031F140F4E130B1F0E230E1F0C03818
:1002F000D1057CF7E4CFE73029F1E83059F1E4305B
:10030000B1F780918000806280938000D0938B0051
:10031000C0938A0004C084B5806884BDC7BDDF91E6
:10032000CF911F91089584B5806284BDC8BDF7CF79
:1003300080918000806880938000D0938900C09372
:100340008800EDCF8091B00080688093B000C093AA
:10035000B300E5CF8091B00080628093B000C0937D
:10036000B400DDCF8E3008F08E50877080648093AB
:100370007C0080917A00806480937A0080917A007A
:1003800086FDFCCF809178009091790008951F92AE
:100390000F920FB60F9211242F933F938F939F9339
:1003A000AF93BF9380912E0190912F01A0913001C6
:1003B000B091310130912D0123E0230F2D3758F5F5
:1003C0000196A11DB11D20932D0180932E019093C4
:1003D0002F01A0933001B0933101809129019091B8
:1003E0002A01A0912B01B0912C010196A11DB11DF4
:1003F0008093290190932A01A0932B01B0932C01A3
:10040000BF91AF919F918F913F912F910F900FBE10
:100410000F901F90189526E8230F0296A11DB11D7D
:10042000D2CFCF93DF9300D000D000D0CDB7DEB7CE
:10043000789484B5826084BD84B5816084BD85B5BF
:10044000826085BD85B5816085BD80916E008160CB
:1004500080936E0010928100809181008260809371
:100460008100809181008160809381008091800073
:100470008160809380008091B10084608093B1009E
:100480008091B00081608093B00080917A00846098
:1004900080937A0080917A00826080937A008091C4
:1004A0007A00816080937A0080917A0080688093DE
:1004B0007A001092C10061E08BE00E94240161E0AB
:1004C00089E00E94240161E083E00E94240162E04F
:1004D00084E00E94240183E28093B00081E0809355
:1004E000B10082E88093800089E1809381008FEFE2
:1004F00090E0909387008093860080911001909106
:100500001101A0911201B091130180930C019093FD
:100510000D01A0930E01B0930F0104E311E040E040
:10052000242E40E0342E8FB7F89420912E01309184
:100530002F01409130015091310129833A834B833F
:100540005C838FBF8EE00E94B201BC01990F880BC3
:10055000990B0E94450720E030EC4FE754E40E94DD
:100560009B069B01AC0160E070E088EC92E40E9485
:1005700067082FE632E143E85AE30E94FA072B01AD
:100580003C01409204015092050160920601709274
:10059000070180E10E94B2016C0183E10E94B20177
:1005A0007C01B601DD0C880B990B0E94450720E009
:1005B00030EC4FE754E40E949B064B015C01B7010D
:1005C000FF0C880B990B0E94450720E030EC4FE7A9
:1005D00054E40E949B069B01AC01C501B4010E943A
:1005E0002A066B017C0120E030E0A9010E949606FA
:1005F00087FD32C120E030E040E85FE3C701B6018B
:100600000E94F507181634F4C12CD12C30E8E32EE3
:100610003FE3F32EC0922501D0922601E0922701FC
:10062000F09228018FE00E94B201BC01990F880B63
:10063000990B0E94450720E030EC4FE754E40E94FC
:100640009B062DEC3CEC4CE45FE30E94FA072DEC9A
:100650003CEC4CEC5EE30E94290660932101709310
:100660002201809323019093240181E10E94B20131
:10067000BC01990F880B990B0E94450720E030ECD4
:100680004FE754E40E949B062FE832EC45E75CE319
:100690000E94FA079B01AC016BE37FED8FE79FE3BC
:1006A0000E9429064B015C0128E431EE4AE75FE332
:1006B0000E94960687FDD4C02BE33FED4FE75FE332
:1006C000C501B4010E94F507181644F42BE3822EED
:1006D0002FED922E2FE7A22E2FE3B22E8092000153
:1006E00090920101A0920201B0920301F80184915D
:1006F000E0E2F1E0F491FE83ECE0F1E0F491FD83BF
:10070000FF2389F081110E94CD002D81E22FF0E0BE
:10071000EE0FFF1FE651FF4FA591B4918C913E81E2
:10072000382381E009F480E010921F01109220012B
:1007300090911E01891771F080931E0189819A8121
:10074000AB81BC818093190190931A01A0931B0186
:10075000B0931C018091190190911A01A0911B0185
:10076000B0911C0129813A814B815C81281B390B96
:100770004A0B5B0BDA01C90140911501509116013A
:100780006091170170911801481759076A077B0794
:10079000B0F490911D0180911E01981781F0809313
:1007A0001D01911103C021E0813009F020E0209368
:1007B0001F01913009F4811190E090932001809104
:1007C0002001882331F08091140131E08327809348
:1007D000140180911401882309F4F9C00E946E0568
:1007E00028EC30E040E050E00E94C60564567109F4
:1007F000810991090E94450720E030E048EC52E46D
:100800000E949B06A70196010E94FA07A30192018C
:100810000E94FA07209110013091110140911201BC
:10082000509113010E942A0624EA30E74DE75FE366
:100830000E94FA076B017C0120E030E0A9010E94D0
:10084000960687FD16C0C0921001D0921101E09269
:100850001201F092130115C0C12CD12C7601DACE11
:1008600098E4892E91EE992E9AE7A92E9FE3B92E4E
:1008700035CF1092100110921101109212011092B6
:10088000130120E030E040E85FE3609110017091D7
:10089000110180911201909113010E94F507181621
:1008A00064F480E090E0A0E8BFE3809310019093AF
:1008B0001101A0931201B0931301C0900001D090D8
:1008C0000101E0900201F09003014090100150906E
:1008D0001101609012017090130120910C01309170
:1008E0000D0140910E0150910F01C701B6010E9408
:1008F000FA074B015C01A701960160E070E080E817
:100900009FE30E942906A30192010E94FA079B011E
:10091000AC01C501B4010E942A066B017C01C092A2
:100920000C01D0920D01E0920E01F0920F01809027
:10093000210190902201A0902301B0902401A501F3
:100940009401C301B2010E942A0620E030E04FE783
:1009500053E40E94FA070E940D077A8369836F3F70
:10096000710529F024F08FEF90E09A838983A981A3
:10097000BA81B7FF02C01A82198269817A818BE03D
:100980000E945501A5019401C701B6010E942A06E3
:1009900020E030E04FE753E40E94FA070E940D0781
:1009A0006F3F710519F014F06FEF70E077FF02C030
:1009B00070E060E089E00E945501B981B093B40015
:1009C0002114310409F4AFCD0E940000ACCD0E9487
:1009D0006E0528EC30E040E050E00E94C605645609
:1009E0007109810991090E94450720E030E048EC37
:1009F00052E40E949B06A70196010E94FA07A301F8
:100A000092010E94FA07209110013091110140914A
:100A10001201509113010E942A060CCFE5E1F1E08A
:100A200082E390E0A0E0B0E080839183A283B3836F
:100A3000148215821682178281E080878187128650
:100A4000138608958F929F92AF92BF92CF92DF92BA
:100A5000EF92FF92CF93DF93EC01688179818A81D5
:100A60009B81611571058105910521F464E279EDA1
:100A70008BE597E02DE133EF41E050E00E94C605A1
:100A800049015A019B01AC01A7EAB1E40E94E505C6
:100A90006B017C01ACEEB4EFA50194010E94F3055B
:100AA000C60ED71EE81EF91EF7FE06C081E0C81A62
:100AB000D108E10880E8F80AC882D982EA82FB827C
:100AC000C701B6019F77DF91CF91FF90EF90DF9044
:100AD000CF90BF90AF909F908F9008958F929F92EC
:100AE000AF92BF92CF92DF92EF92FF926091080196
:100AF0007091090180910A0190910B0161157105B6
:100B00008105910521F464E279ED8BE597E02DE113
:100B100033EF41E050E00E94C60549015A019B01B4
:100B2000AC01A7EAB1E40E94E5056B017C01ACEEE3
:100B3000B4EFA50194010E94F305C60ED71EE81E6E
:100B4000F91EF7FE06C081E0C81AD108E10880E866
:100B5000F80AC0920801D0920901E0920A01F092CD
:100B60000B01C701B6019F77FF90EF90DF90CF9008
:100B7000BF90AF909F908F900895609308017093FD
:100B8000090180930A0190930B010895052E97FBAC
:100B90001EF400940E94DD0557FD07D00E94F80561
:100BA00007FC03D04EF40C94DD055095409530952C
:100BB00021953F4F4F4F5F4F0895909580957095C9
:100BC00061957F4F8F4F9F4F08950E941A06A59FF2
:100BD000900DB49F900DA49F800D911D1124089538
:100BE000B7FF0C94E5050E94E505821B930B089561
:100BF000A1E21A2EAA1BBB1BFD010DC0AA1FBB1F21
:100C0000EE1FFF1FA217B307E407F50720F0A21B92
:100C1000B30BE40BF50B661F771F881F991F1A94FF
:100C200069F760957095809590959B01AC01BD0129
:100C3000CF010895A29FB001B39FC001A39F700D83
:100C4000811D1124911DB29F700D811D1124911DD4
:100C500008955058BB27AA270E9441060C94BB0751
:100C60000E94AD0738F00E94B40720F039F49F3F8E
:100C700019F426F40C94AA070EF4E095E7FB0C9403
:100C8000A407E92F0E94CC0758F3BA17620773072D
:100C90008407950720F079F4A6F50C94EE070EF47E
:100CA000E0950B2EBA2FA02D0B01B90190010C017C
:100CB000CA01A0011124FF27591B99F0593F50F494
:100CC000503E68F11A16F040A22F232F342F4427EC
:100CD000585FF3CF469537952795A795F0405395E4
:100CE000C9F77EF41F16BA0B620B730B840BBAF0B4
:100CF0009150A1F0FF0FBB1F661F771F881FC2F71F
:100D00000EC0BA0F621F731F841F48F48795779532
:100D10006795B795F7959E3F08F0B0CF9395880FEC
:100D200008F09927EE0F9795879508950E94800700
:100D300008F481E008950E94AF060C94BB070E945E
:100D4000B40758F00E94AD0740F029F45F3F29F046
:100D50000C94A40751110C94EF070C94AA070E945D
:100D6000CC0768F39923B1F3552391F3951B550BE9
:100D7000BB27AA2762177307840738F09F5F5F4F6E
:100D8000220F331F441FAA1FA9F335D00E2E3AF0AD
:100D9000E0E832D091505040E695001CCAF72BD0C5
:100DA000FE2F29D0660F771F881FBB1F2617370716
:100DB0004807AB07B0E809F0BB0B802DBF01FF2748
:100DC00093585F4F3AF09E3F510578F00C94A4077A
:100DD0000C94EF075F3FE4F3983ED4F38695779544
:100DE0006795B795F7959F5FC9F7880F911D969501
:100DF000879597F90895E1E0660F771F881FBB1F5D
:100E0000621773078407BA0720F0621B730B840B09
:100E1000BA0BEE1F88F7E09508950E9414076894B6
:100E2000B1110C94EF0708950E94D40788F09F57E2
:100E300098F0B92F9927B751B0F0E1F0660F771FFE
:100E4000881F991F1AF0BA95C9F714C0B13091F0F4
:100E50000E94EE07B1E008950C94EE07672F782FFB
:100E60008827B85F39F0B93FCCF3869577956795B9
:100E7000B395D9F73EF490958095709561957F4F25
:100E80008F4F9F4F0895E89409C097FB3EF49095CB
:100E90008095709561957F4F8F4F9F4F9923A9F053
:100EA000F92F96E9BB279395F695879577956795E2
:100EB000B795F111F8CFFAF4BB0F11F460FF1BC026
:100EC0006F5F7F4F8F4F9F4F16C0882311F096E9B9
:100ED00011C0772321F09EE8872F762F05C0662367
:100EE00071F096E8862F70E060E02AF09A95660F20
:100EF000771F881FDAF7880F9695879597F90895D9
:100F0000990F0008550FAA0BE0E8FEEF161617061A
:100F1000E807F907C0F012161306E407F50798F082
:100F2000621B730B840B950B39F40A2661F0232B9B
:100F3000242B252B21F408950A2609F4A140A69517
:100F40008FEF811D811D089597F99F6780E870E0FC
:100F500060E008959FEF80EC089500240A9416162F
:100F6000170618060906089500240A941216130697
:100F7000140605060895092E0394000C11F4882325
:100F800052F0BB0F40F4BF2B11F460FF04C06F5F41
:100F90007F4F8F4F9F4F089557FD9058440F551F17
:100FA00059F05F3F71F04795880F97FB991F61F0EB
:100FB0009F3F79F087950895121613061406551F62
:100FC000F2CF4695F1DF08C0161617061806991FCE
:100FD000F1CF86957105610508940895E894BB27C3
:100FE00066277727CB0197F908950E94800708F4B8
:100FF0008FEF08950E940D080C94BB070E94AD0767
:1010000038F00E94B40720F0952311F00C94A40747
:101010000C94AA0711240C94EF070E94CC0770F3DC
:10102000959FC1F3950F50E0551F629FF001729F8D
:10103000BB27F00DB11D639FAA27F00DB11DAA1F9C
:10104000649F6627B00DA11D661F829F2227B00DE9
:10105000A11D621F739FB00DA11D621F839FA00D74
:10106000611D221F749F3327A00D611D231F849FC4
:10107000600D211D822F762F6A2F11249F5750401B
:101080009AF0F1F088234AF0EE0FFF1FBB1F661F96
:10109000771F881F91505040A9F79E3F510580F05F
:1010A0000C94A4070C94EF075F3FE4F3983ED4F34D
:1010B000869577956795B795F795E7959F5FC1F703
:1010C000FE2B880F911D9695879597F90895FA0143
:1010D000EE0FFF1F309621053105A1F16115710555
:1010E00061F48038BFE39B0749F16894903881052B
:1010F00061F08038BFEF9B0741F099234AF5FF3F2D
:10110000E1053105210519F1E8940894E795D90125
:10111000AA2329F4AB2FBE2FF85FD0F310C0FF5FD6
:1011200070F4A695E0F7F73950F019F0FF3A38F46B
:101130009F779F930DD00F9007FC9058089546F02D
:101140000C94AA0760E070E080E89FE308954FE701
:101150009F775F934F933F932F930E9462092F9144
:101160003F914F915F910E94FA070C94BF0829F4B8
:1011700016F00C94A4070C94EE070C94AA070E9496
:10118000D407A8F39638A0F707F80F92E8942BE35A
:101190003AEA48EB5FE70E9410080F920F920F9215
:1011A0004DB75EB70F920E94AA09E8E6F0E00E94F0
:1011B000F1084F915F91EF91FF91E595EE1FFF1FB1
:1011C00049F0FE57E0684427EE0F441FFA95E1F717
:1011D0004195550B0E9424090F9007FE0C941809A5
:1011E0000895DF93CF931F930F93FF92EF92DF92B7
:1011F0007B018C01689406C0DA2EEF010E940D0875
:10120000FE01E894A5912591359145915591A6F35C
:10121000EF010E944106FE019701A801DA9469F7E7
:10122000DF90EF90FF900F911F91CF91DF91089584
:101230009B01AC0160E070E080E89FE30C949B06AA
:101240000C94A4070C94DE090E94D407D8F39923C8
:10125000C9F3940F511DA3F39150504094F059F0ED
:10126000882332F0660F771F881F91505040C1F7D6
:101270009E3F51052CF7880F911D9695879597F9FC
:1012800008955F3FACF0983E9CF0BB27869577951C
:101290006795B79508F4B1609395C1F7BB0F58F700
:1012A00011F460FFE8CF6F5F7F4F8F4F9F4FE3CF09
:1012B0000C94EF0716F00C94DE090C94AA076894BE
:1012C0000C94A4070E94D407A8F39923C1F3AEF3AA
:1012D000DF93CF931F930F93FF92C92FDD278823AE
:1012E0002AF02197660F771F881FDAF720E030E099
:1012F00040E85FEB9FE3883920F0803E38F021968C
:101300008F770E942A06E0E9F0E004C00E942A06D6
:10131000EDEBF0E00E94F1088B01BE01EC01FB2E29
:101320006F5771097595771F880B990B0E944507B8
:1013300028E132E741E35FE30E940D08AF2D9801F9
:10134000AE01FF900F911F91CF91DF910E94410656
:101350000C94BB07FA01DC01AA0FBB1F9B01AC0177
:10136000BF5728F4222733274427507820C0B7518D
:1013700090F4AB2F0024469537952795011CA39533
:10138000D2F3002071F0220F331F441FB395DAF31C
:101390000ED00C94290661307105A0E88A07B94681
:1013A00030F49B01AC016627772788279078309628
:1013B00021F0208331834283538308959F3F31F08E
:1013C000915020F4879577956795B795880F911D73
:1013D0009695879597F90895EE0FFF1F0590F49164
:0813E000E02D0994F894FFCF01
:0C13E8003BDF7F3F6F12833A01000000E2
:00000001FF
